:020000040000FA
:100000008316FF30853000308600C13081008312B6
:1000100003018501860191018D019201FF308C0061
:10002000930094009500E7308100051E012B010824
:10003000031D1728E73081008D0A03198C0A14303C
:100040000C020319002885192D281408031D3528D2
:10005000FF309400861793014E28140803193528A1
:10006000861394011728950317281208031D4728A3
:100070001508031D33281308031D172806148615B9
:100080000611FF309200930002308E0017288E0B6D
:100090001728061086110615920117280C08031D53
:1000A0005A280D08263A0319862826300D02031C0B
:1000B00086286B280C08013A0319632801300C02CA
:1000C000031882286B280D08903A03198228903073
:1000D0000D020318822825308D02031C8C030310A7
:1000E0008C0C8D0C03108C0C8D0C743091000D0851
:1000F00011020A108A1400228F008C018D010F0852
:100100009500172832308F0086107D288F018614C5
:020110007D2848
:10040000820732343134313430342F342F342E34A7
:100410002E342D342D342C342C342B342B342A34DC
:100420002A342934293428342834273427342634EC
:1004300026342534253424342434233423342234FC
:10044000223421342134203420341F341F341F340B
:100450001E341E341D341D341C341C341B341B3418
:100460001A341A3419341934193418341834173426
:100470001734163416341534153414341434143433
:10048000133413341234123411341134113410343F
:1004900010340F340F340E340E340D340D340D344B
:1004A0000C340C340B340B340A340A340A34093457
:1004B0000934083408340734073407340634063462
:1004C000053405340434043404340334033402346E
:1004D0000234023401340134003400340034003476
:0E04E00032343234323432343234323408346E
:10060000002886148613851D062B122B8617E730CB
:10061000960004309700960B0E2B970B0B2B102B8C
:100620001E2B012B86175F309600EB309700960B40
:100630001A2B970B172B1C2B1E2B012B06140611A4
:100640008F30960002309700960B272B970B242BA8
:08065000292B06100615012BF1
:02400E00F23F7F
:00000001FF
